:100000000C9463000C948B000C948B000C948B006C
:100010000C94C21C0C948B000C948B000C94661CEA
:100020000C948B000C948B000C948B000C948B0024
:100030000C948B000C948B000C948B000C948B0014
:100040000C941C1C0C948B000C948B000C948B0057
:100050000C948B000C948B000C948B000C948B00F4
:100060000C941A1D0C948B00000000002400270043
:100070002A000000000023002600290000000008DC
:10008000000201000003040700000000000000005F
:10009000010204081020408001020408102001021F
:1000A0000408102000000000250028002B00040494
:1000B0000404040404040202020202020303030310
:1000C00003030200391E11241FBECFEFD8E0DEBFAC
:1000D000CDBF14E0A0E0B1E0E8EAF4E502C005908D
:1000E0000D92A835B107D9F726E0A8E5B4E001C024
:1000F0001D92A232B207E1F710E0C3E6D0E004C0DF
:100100002197FE010E94062AC236D107C9F70E9434
:10011000B81E0C94522A0C9400008230910538F0DD
:10012000880F991F880F991F05970197F1F7089578
:100130008091220120E4829FC00111248760809376
:100140007C0080917A00806480937A0080917A00AC
:1001500086FDFCCF809178009091790008952091E0
:10016000BD0581E0213208F044C0809199058111DC
:10017000FCCF8091BC0592E09093990591E090931B
:1001800098059FEF909397051092960520939505FB
:10019000ACE9B5E0E5E7F5E090E0291331C0109255
:1001A000740590917405880F892B80937405809154
:1001B0007305813049F51092730580917405809321
:1001C000BB008091BC0083FDF8CF85EC8093BC0020
:1001D000809199058230E1F3809197058F3FB1F0CE
:1001E000809197058032A1F080919705803391F03E
:1001F00084E010929B051092BD0510929A05089517
:100200003D9131939F5FC9CF85EEE0CF80E0F1CF84
:1002100082E0EFCF83E0EDCF833081F028F48130AE
:1002200099F08230A9F008958730A9F08830C9F09C
:100230008430B1F4809180008F7D03C08091800074
:100240008F7780938000089584B58F7784BD08955B
:1002500084B58F7DFBCF8091B0008F778093B00005
:1002600008958091B0008F7DF9CFCF93DF93282F31
:1002700030E0F901E458FF4F8491F901E057FF4F56
:10028000D491F901E255FF4FC491CC23A1F0811123
:100290000E940C01EC2FF0E0EE0FFF1FEE58FF4F15
:1002A000A591B491EC91ED2381E090E009F480E018
:1002B000DF91CF91089580E090E0FACF1F93CF9324
:1002C000DF93282F30E0F901E458FF4F8491F901C2
:1002D000E057FF4FD491F901E255FF4FC491CC2371
:1002E000A9F0162F81110E940C01EC2FF0E0EE0F07
:1002F000FF1FEC55FF4FA591B4918FB7F894EC9187
:10030000111108C0D095DE23DC938FBFDF91CF9110
:100310001F910895DE2BF8CFCF93DF9390E0FC017F
:10032000E057FF4F249182559F4FFC018491882311
:10033000C9F090E0880F991FFC01E859FF4FA59183
:10034000B491FC01EC55FF4FC591D49161110DC0E2
:100350009FB7F8948C91209582238C9388812823D1
:1003600028839FBFDF91CF910895623051F49FB7EA
:10037000F8943C91822F809583238C93E8812E2BD7
:10038000EFCF8FB7F894EC912E2B2C938FBFEACF41
:100390008F929F92AF92BF92CF92DF92EF92FF9295
:1003A000CF936C0180912301853069F08F3F09F470
:1003B00070C0CF91FF90EF90DF90CF90BF90AF9043
:1003C0009F908F900895E2ECF0E0C491C7FDF1CFCB
:1003D00061E085E00E948C01CC2319F0C23009F065
:1003E00022C1F12CE12C60E072E18AE790E0A701E4
:1003F00096010E948F2949015A01DA01C90101972A
:10040000A109B1098F3F9105A105B10509F00CF4CF
:10041000EEC060E472E48FE090E0A70196010E94D4
:100420008F292150310941095109C23009F0A0C07A
:1004300082E02F3F31054105510509F00CF488C1D8
:1004400060E970ED83E090E0A70196010E948F299A
:10045000215031094109510983E02F3F3105410500
:10046000510509F00CF474C168E478EE81E090E085
:10047000A70196010E948F29215031094109510994
:100480002F3F31054105510511F00CF08FC084E07C
:100490005FC185E080932301E2ECF0E0C491CF3F9F
:1004A00009F487CFC13021F150F0C23009F43EC0C9
:1004B000C7FD7FCF61E085E00E948C018FCF14BC27
:1004C00015BC84B5826084BD85B5816085BDE3EBD4
:1004D000F0E0E491F0E0EE0FFF1FEC55FF4F859147
:1004E0009491E5E9F0E0E491E093C205C0E070CFBB
:1004F000109280001092810080918100886080932A
:10050000810080918100816080938100E3EBF0E0C5
:10051000E491F0E0EE0FFF1FEC55FF4F85919491B1
:10052000E5E9F0E0E491E093C10552CF1092B0000C
:100530001092B1008091B00082608093B0008091F1
:10054000B10081608093B100E3EBF0E0E491F0E072
:10055000EE0FFF1FEC55FF4F859194919093C005CE
:100560008093BF05E5E9F0E0E491E093BE0530CF6C
:100570002F3F31054105510509F00CF452C068E4E4
:1005800078EE81E090E0A70196010E948F2921502A
:10059000310941095109CC2309F4AFC02F3F31057E
:1005A0004105510511F00CF0B0C071CF64E274EF59
:1005B00080E090E0A70196010E948F292150310927
:1005C0004109510985E02F3F31054105510509F0E9
:1005D00008F4BEC062E17AE780E090E0A7019601EE
:1005E0000E948F2921503109410951099CC09C0169
:1005F00081E0C111ADC095B5987F892B85BD27BD20
:100600008FEF9FEFDC018093CB059093CC05A093F7
:10061000CD05B093CE0580916E00826080936E0010
:10062000C8CE82E0E6CFF12CE12C60E072E18AE7EF
:1006300090E0A70196010E948F29215031094109BC
:10064000510991E02115310581E0480751056CF011
:1006500068E478EE81E090E0A70196010E948F297E
:10066000215031094109510993E0C13009F076C0A8
:1006700080918100887F892B80938100309389004D
:10068000209388008FEF9FEFDC018093C705909344
:10069000C805A093C905B093CA0580916F00826018
:1006A00080936F0086CE2093B3008FEF9FEFDC0125
:1006B0008093C3059093C405A093C505B093C60568
:1006C0008091700082608093700073CE84E02F3F31
:1006D00031054105510509F008F48DCF9AE0B59434
:1006E000A794979487949A95D1F7A50194012150E6
:1006F00031094109510985E07ECF83E02F3F310563
:100700004105510509F00CF476CF62E17AE780E00B
:1007100090E0A70196010E948F29215031094109DB
:100720005109CC2399F286E02F3F3105410551054F
:1007300079F070F08AE0B594A794979487948A959D
:10074000D1F7A5019401215031094109510987E0F0
:100750009091B100987F892B8093B100C13009F44A
:100760008DCFC23009F49FCFC11123CE48CF3FB700
:10077000F89480916F0590917005A0917105B091EA
:10078000720526B5A89B05C02F3F19F00196A11D43
:10079000B11D3FBFBA2FA92F982F8827BC01CD01CB
:1007A000620F711D811D911D42E0660F771F881F2A
:1007B000991F4A95D1F708958F929F92AF92BF9259
:1007C000CF92DF92EF92FF926B017C010E94B70300
:1007D0004B015C01C114D104E104F104B9F00E94A1
:1007E000B703681979098A099B09683E7340810536
:1007F000910580F321E0C21AD108E108F10888EEE2
:10080000880E83E0981EA11CB11CE4CFFF90EF90EE
:10081000DF90CF90BF90AF909F908F9008952FB7AB
:10082000F89460916B0570916C0580916D059091C5
:100830006E052FBF089581E0809384040895089584
:10084000089508959091230189130BC0E2ECF0E024
:10085000E4919FEF90932301E13049F028F0E230DA
:1008600061F060E00C945E0110926E00FACF9091FE
:100870006F009D7F90936F00F4CF909170009D7FEB
:100880009093700091E09093B0009091B100987FA8
:1008900094609093B1001092B300E3CFAF92BF92F7
:1008A000CF92DF92EF92FF920F931F93CF93DF933C
:1008B0006C017B018B01040F151FEB015E01AE186B
:1008C000BF08C017D10759F06991D601ED91FC918D
:1008D0000190F081E02DC6010995892B79F7C501BA
:1008E000DF91CF911F910F91FF90EF90DF90CF900C
:1008F000BF90AF900895089585ED8093BC008091DE
:10090000BC0084FDFCCF1092990508952091DD0470
:10091000260F3327331F21323105ECF4209199053E
:10092000FC0190E080E0243069F082E00895A0911D
:10093000DD042191AC0143545B4FA40FB52FB11DD1
:100940002C930196861798F38091DD04680F6093CD
:10095000DD0480E0089581E008950895E0910805A0
:1009600080910705E81730F4F0E0E356FB4F8081F3
:1009700090E008958FEF9FEF089590910805809182
:1009800007052FEF3FEF981748F4E92FF0E0E35603
:10099000FB4F208130E09F5F90930805C9010895C7
:1009A0008091070590910805891B990B0895CF92B6
:1009B000DF92EF92FF920F931F93CF93DF937C010F
:1009C000CB018A0120919A05222389F0EB016B016A
:1009D000C40ED51ECC15DD0569F06991D701ED91E6
:1009E000FC910190F081E02DC7010995F3CF642FB0
:1009F0000E948604C801DF91CF911F910F91FF9053
:100A0000EF90DF90CF900895CF93DF931F92CDB7F3
:100A1000DEB7698320919A052223F9F02091BD0564
:100A2000203258F021E030E0FC013383228390E053
:100A300080E00F90DF91CF91089580919B05E82F82
:100A4000F0E0E456FA4F998190838F5F80939B0585
:100A50008093BD0581E090E0ECCF61E0CE0101968E
:100A60000E948604F7CF0F931F93CF93DF938B01E0
:100A700091E090939A0590E69093BC0510929B05A7
:100A80001092BD05682F8FEC95E00E940405E801E7
:100A900019E0115031F069918FEC95E00E94040546
:100AA000F8CFDF91CF911F910F910C94AF0090E0A0
:100AB00080E008950F931F93CF9360E082E00E943F
:100AC0005E0180919C0490E0499620912006821B53
:100AD00091090E948D008FE00E943501C09196041B
:100AE000892B09F48CC00E940F04609397047093C3
:100AF00098048093990490939A04C1111EC00E9497
:100B00000F04009192041091930420919404309169
:100B10009504601B710B820B930B6230710581058C
:100B2000910558F081E08093960410928E04109203
:100B30008F04109290041092910461E082E00E9470
:100B40005E0183EC90E00197F1F760E082E00E94A3
:100B50005E0180919B0490E0499620912006821BC3
:100B600091090E948D0083E00E943501C0918904A3
:100B7000892B09F468C00E940F0460938A04709363
:100B80008B0480938C0490938D04C1111EC00E942D
:100B90000F04009185041091860420918704309100
:100BA0008804601B710B820B930B62307105810509
:100BB000910558F081E08093890410928E04109280
:100BC0008F04109290041092910461E082E00E94E0
:100BD0005E0183EC90E00197F1F780911606823078
:100BE00011F0843041F4809189049091960490939F
:100BF000890480939604CF911F910F9108950E94CC
:100C00000F046093920470939304809394049093E0
:100C10009504CC2309F491CF0E940F04009197040E
:100C2000109198042091990430919A04601B710BE3
:100C3000820B930B6B3071058105910508F47DCF14
:100C4000109296047ACF0E940F04609385047093EB
:100C500086048093870490938804CC2309F4B5CF4D
:100C60000E940F0400918A0410918B0420918C043F
:100C700030918D04601B710B820B930B6B307105EF
:100C80008105910508F4A1CF109289049ECFCF92DF
:100C9000DF92EF92FF92CF93C4E6C12CD12C760164
:100CA00080918404882361F01092840480914C0523
:100CB00090914D05CF91FF90EF90DF90CF900895E8
:100CC0000E949800092E000CAA0BBB0BC80ED91E5F
:100CD000EA1EFB1EC15021F7C701B6016B5F7F4FB3
:100CE0008F4F9F4F2AE030E040E050E00E94C12942
:100CF000A0E1B7E20E94AE2926EF37E240E050E0E3
:100D00000E94C129C901D6CFCF92DF92EF92FF9204
:100D10000F931F93CF93DF938C01D42FC0E06B010F
:100D2000770FEE08FF08C8010E94C801C701B6018D
:100D30000E94DC0385E00E942204C701B6010E94E4
:100D4000DC03CF5FDC13EFCFDF91CF911F910F91C9
:100D5000FF90EF90DF90CF900895CF93C62F91E052
:100D600090939A0590E69093BC0510929B05109283
:100D7000BD05682F8FEC95E00E9404056C2F8FEC69
:100D800095E00E940405CF910C94AF004F925F92C2
:100D90006F927F928F929F92AF92BF92CF92DF928B
:100DA000EF92FF921F93CF93DF93CDB7DEB72897D3
:100DB0000FB6F894DEBF0FBECDBF6B017C01109162
:100DC0002101DC01CB018052914AA740B109813257
:100DD0009449A747B640F0F0146010932101609148
:100DE000210183E00E94AD0628960FB6F894DEBF7D
:100DF0000FBECDBFDF91CF911F91FF90EF90DF909D
:100E0000CF90BF90AF909F908F907F906F905F90AA
:100E10004F90089560911D0170911E0180911F01F6
:100E200090912001A70196010E94C12949015A0110
:100E30002601370144245524E0EF6E224528462838
:100E4000472849F09695879577956795F694E794A6
:100E5000D794C794EDCF27E0660F771F881F991F9F
:100E60002A95D1F7A70196010E94C129E7E0880CD5
:100E7000991CAA1CBB1CEA95D1F7E2E09E1AA108B6
:100E8000B108820E931EA41EB51ED982CA82AB82FF
:100E90009C828D82F4E0CC0CDD1CEE1CFF1CFA95CC
:100EA000D1F7CC24DD2420EFE222FF24E82AEE82D1
:100EB0007F836887BE016F5F7F4F8AE30E9433059F
:100EC00060911C016C6082E10E94AD061B7F85CFA2
:100ED000FF920F931F93CF93DF9303EF15E0D0E0C2
:100EE000C0E0F801F1908F01CE010E947929F81637
:100EF00021F06F2DCE010E9481292196CF32D1059C
:100F000081F783EF95E0DF91CF911F910F91FF90D3
:100F10000895CF93DF93EC0160E08E810E945E0123
:100F200061E08E810E945E0160E08E810E945E0120
:100F30008BE891E00197F1F7DF91CF910895CF927F
:100F4000DF92EF92FF920F931F93CF93DF936C0189
:100F50007C0187E0E80EF11CD0E0C0E0062F10E035
:100F6000B8010C2E02C0759567950A94E2F761707E
:100F7000F70181917F010E945E012196C430D10565
:100F800079F7C601DF91CF911F910F91FF90EF90FC
:100F9000DF90CF900C948907CF92DF92EF92FF926F
:100FA0000F931F93CF93DF93EC01F62E642F8C8168
:100FB0000E945E018D818F3F19F060E00E945E010A
:100FC0000F2D10E08F8584FF25C06E0187E0C80ECD
:100FD000D11CF12CE12CB8010E2C02C0759567953F
:100FE0000A94E2F76170F60181916F010E945E013F
:100FF000FFEFEF1AFF0A88E0E816F10461F7CE016F
:10100000DF91CF911F910F91FF90EF90DF90CF90E4
:101010000C948907B80184E0759567958A95E1F786
:10102000CE010E949F076F2DCE01DF91CF911F91BE
:101030000F91FF90EF90DF90CF900C949F0740E0CE
:10104000682F8BED95E00C94CC07CF93DF93823023
:1010500029F49091EA0598609093EA058093EE0553
:101060001092EF0580E48093F00580E18093F10514
:1010700080E58093F20561E08091DF050E948C019C
:101080008091E0058F3F19F061E00E948C0161E0E2
:101090008091E1050E948C01CBEDD5E09E012B5D96
:1010A00035408091EA0584FD0BC084E090E02196F4
:1010B0002817390744F461E08E810E948C01EECF3D
:1010C00088E090E0F4CF8BE39DE00197F1F760E0DA
:1010D0008091DF050E945E0160E08091E1050E9441
:1010E0005E018091E0058F3F19F060E00E945E0193
:1010F0008091EA0584FD39C063E08BED95E00E94A4
:101100009F07CBE4D6E4CE010197F1F763E08BEDC6
:1011100095E00E949F072197F1F763E08BED95E042
:101120000E949F0783E592E00197F1F762E08BED63
:1011300095E00E949F078091EA0580620E941F0847
:1011400084E08093EB058CE00E941F0881E00E9400
:101150001F088BE39FE10197F1F782E08093EC0594
:1011600086E0DF91CF910C941F0880620E941F08D7
:101170008BE496E40197F1F78091EA0580620E9482
:101180001F0883E592E00197F1F78091EA058062FC
:101190000E941F08D0CF41E00E94CC0781E090E080
:1011A0000895EF92FF920F931F93CF93DF93C82F71
:1011B0008B0121E18202C00111249C01285A3B4F7E
:1011C0007901B901C8010E94322A892B79F1EC2FEB
:1011D0008091EE05C81710F0EFEFE80FF0E0E55250
:1011E000FA4F848980680E941F08F801019000204E
:1011F000E9F73197AF01401B510BB8018BED95E03A
:101200000E944E04B801C7010E943B2AE8010990E0
:101210000020E9F72197C01BC03140F441E060E2B3
:101220008BED95E00E94CC07CF5FF6CFDF91CF9199
:101230001F910F91FF90EF90089562E471E080E0BC
:101240000E94D10863E571E081E00E94D1080E940C
:10125000680768EE73E080E090E00C94DC034F9246
:101260005F926F927F928F929F92AF92BF92CF9236
:10127000DF92EF92FF9281E10E943501892B19F4F0
:1012800081E08093820480918204882371F081E15F
:101290000E943501892B49F08091F405823328F4AE
:1012A000109282048F5F8093F40584E00E943501E0
:1012B000892B19F481E08093810480918104882333
:1012C00071F084E00E943501892B49F08091F4058A
:1012D000823028F01092810481508093F40580912F
:1012E0001606833020F180912006882369F08091D2
:1012F0002006811107C110925F05109260051092BF
:1013000061051092620513C0E0910501F09106019C
:1013100080810E943501892B51F70E940F04609350
:101320005F0570936005809361059093620520913D
:10133000F40530E050E040E060EB74E080E090E0E5
:101340000E94C12969017A0140907D0450907E0479
:1013500060907F0470908004411451046104710412
:1013600009F0F3C00E940F0480906305909064051B
:10137000A0906505B0906605681979098A099B09EE
:101380006C157D058E059F0508F0C1C061E086E003
:101390000E945E018091FE059091FF050E94C801A8
:1013A00081E080937C0480918E0490918F04A091C1
:1013B0009004B0919104892B8A2B8B2B09F04FC09C
:1013C00080917D0490917E04A0917F04B09180046F
:1013D000892B8A2B8B2B09F0DEC10E940F04809091
:1013E000630590906405A0906505B0906605681946
:1013F00079098A099B096C157D058E059F0548F4BE
:1014000080912006882309F4B2C1809120068111C1
:10141000E0C10E940F0480905F0590906005A0904D
:101420006105B09062059B01AC01281939094A0990
:101430005B0949015A01A3E0B0E0A70196010E94AF
:10144000AE2986169706A806B90648F480912006AC
:10145000882309F4C3C1809120068111E1C1C090A5
:101460008E04D0908F04E0909004F09091048091CD
:101470002006811108C2C114D104E104F10409F06D
:101480001AC280917D0490917E04A0917F04B09156
:101490008004892B8A2B8B2B09F029C280915A0555
:1014A00081115BC280915905882309F442C2809161
:1014B000F4054AE06AE275E090E00E9413296FE5C6
:1014C00071E089E195E00E943B2A6AE275E089E1DA
:1014D00095E00E94272A69E671E089E195E00E9483
:1014E000272A69E175E081E0FF90EF90DF90CF90CF
:1014F000BF90AF909F908F907F906F905F904F9034
:101500000C94D10880918904811107CFF4CE0E94F8
:101510000F0480905F0590906005A0906105B090E9
:1015200062059B01AC01281939094A095B09490187
:101530005A01A3E0B0E0A70196010E94AE298616E9
:101540009706A806B90608F421CF60E086E00E945D
:101550005E0185E00E94220445284628472851F470
:101560000E940F0460937D0470937E0480937F0437
:10157000909380040E940F0480907D0490907E04DC
:10158000A0907F04B09080042B013C0148185908BA
:101590006A087B08A0910401B0E0A70196010E94AF
:1015A000AE29641575058605970508F0FCCE4091B7
:1015B00063055091640560916505709166058091A1
:1015C0005F0590916005A0916105B0916205481793
:1015D00059076A077B0708F093C080917B04882332
:1015E00081F00E940F0460936305709364058093FB
:1015F00065059093660581E08093590510927B0400
:101600001BC0809120068823D1F080912006811193
:1016100020C090917A04992309F10E940F046093ED
:101620005F0570936005809361059093620581E08A
:101630008093590510927A0480937C043EC0E09117
:101640000201F091030180810E943501892B49F24A
:10165000DCCF909196049111C4CFDBCF882309F49D
:101660003FC080912006811146C080911F068823CB
:1016700019F083E08093040181E080935905809301
:101680007C040E940F049B01AC01281939094A0906
:101690005B0949015A01A0910401B0E0A70196013C
:1016A0000E94AE29681579058A059B0508F07BCE56
:1016B0001092590510927C0481E0809304011092ED
:1016C0007D0410927E0410927F0410928004109288
:1016D0008E0410928F04109290041092910463CEA5
:1016E000E0910501F091060180810E943501892B6E
:1016F00009F493CFB6CF8091890481118ECFB5CFF5
:1017000080917A04811189CF809120068823A1F0ED
:101710008091200681111BC090917B04911161CFB3
:101720008823D1F080912006882309F49ECF8091F0
:101730009604811156CF99CFE0910501F0910601F1
:1017400080810E943501892B09F467CFE1CF909108
:101750008904911162CFE0CFE0910201F091030181
:1017600080810E943501892B09F43BCFDBCFE091CA
:101770000201F091030180810E943501892B09F457
:1017800044CE0E940F0460938E0470938F04809364
:1017900090049093910480917D0490917E04A09197
:1017A0007F04B0918004892B8A2B8B2B09F431CED6
:1017B000809120068823C9F180912006811157C0AD
:1017C000C0908E04D0908F04E0909004F09091042B
:1017D00052CE8091960481111CCED3CFE0910501A9
:1017E000F091060180810E943501892B09F433CEE6
:1017F0000E940F0460938E0470938F048093900472
:101800009093910480917D0490917E04A0917F0437
:10181000B0918004892B8A2B8B2B09F420CEC8CF62
:101820008091890481111BCEE3CFE0910201F091F8
:10183000030180810E943501892B09F4BDCF80917D
:10184000200681112EC0E0910501F09106018081F2
:101850000E943501892B29F10E940F0460938E04A8
:1018600070938F048093900490939104F8CD8091AD
:101870009604882321F3C0908E04D0908F04E090CA
:101880009004F0909104CD28CE28CF2809F406CEFC
:1018900080919604811125C080918904811143C0F3
:1018A000FDCD80912006882309F48ACF8091890498
:1018B0008111E1CFD1CF0E940F046C197D098E09EF
:1018C0009F09663071058105910508F4DACDE09134
:1018D0000201F091030180810E943501892B09F0FA
:1018E000D0CD81E080937B0410927A04D7CDC114CF
:1018F000D104E104F10409F4D1CD0E940F046C1964
:101900007D098E099F09603171058105910508F4F3
:10191000C5CDE0910501F091060180810E9435015D
:10192000892B09F0BBCD81E080937A0410927B046F
:10193000B5CD80915C056EE671E08111D4CD8091CA
:101940005E056DE771E08A300CF0CDCD1092350563
:101950001092340568E672E0C6CDFF90EF90DF90FC
:10196000CF90BF90AF909F908F907F906F905F903F
:101970004F9008950F931F93CF93DF93E9E1F5E024
:1019800081E1DF011D928A95E9F7EAE2F5E08AE05C
:10199000DF011D928A95E9F700914E0510914F05E0
:1019A000209150053091510580915C05811105C051
:1019B00080916905883009F07EC080915205909130
:1019C0005305092E000CAA0BBB0BBC01CD01600F07
:1019D000711F821F931F2AE04AE255E00E942D29C1
:1019E00068E672E089E195E00E943B2ACAE2D5E010
:1019F00009900020E9F7CB52D540DD278E01065033
:101A00001109A8016AE275E089E195E00E94422A85
:101A10006DE571E089E195E00E94272AB801665DD5
:101A20007A4F43E050E089E195E00E94422A6DE55B
:101A300071E089E195E00E94272ABE01695D7A4F35
:101A400080915C05811106C08091690541E050E0FC
:101A5000883011F443E050E089E195E00E94422A89
:101A600080915805813009F442C0D0F1823009F4E8
:101A700041C0833009F441C080916705882331F06B
:101A800080915A056EE971E0882331F080910B0650
:101A9000882331F062EA71E089E195E00E94272A0B
:101AA0001092290569E175E080E0DF91CF911F91E7
:101AB0000F910C94D108C901B8016E5C7F4F8F4F14
:101AC0009F4F2AE04AE255E00E942D2980910A06A4
:101AD0006EE871E0882309F485CF61E971E082CF77
:101AE0006FE973E089E195E00E94272AC5CF6FEA8C
:101AF00073E0F8CF64E971E0F5CF69E971E0F2CF06
:101B0000AF92BF92CF92DF92FF920F931F93CF932A
:101B1000DF9360E08FE00E948C0160E083E00E9430
:101B20008C0110929C0493ECC92ED12CD0919C0472
:101B3000DF5FD0939C0410E000E0C0E0AD2EB12C3C
:101B400061E082E00E945E01C6010197F1F760E06A
:101B500082E00E945E01C5010E948D008FE00E941C
:101B60003501892B19F004E610E0C1E00F5F1F4F2B
:101B7000043611052CF3CC2311F0DF3FB9F6109297
:101B80009B0483ECC82ED12CC0919B04CF5FC093E3
:101B90009B0410E000E0F12CAC2EB12C61E082E05F
:101BA0000E945E01C6010197F1F760E082E00E94A9
:101BB0005E01C5010E948D0083E00E943501892BE2
:101BC00021F004E610E0FF24F3940F5F1F4F04366A
:101BD000110524F3FF2069F1CF3FB1F61092070100
:101BE0001092200666EA71E080E00E94D10864EB62
:101BF00071E081E00E94D10860ED77E080E090E044
:101C00000E94DC030E94BA0C80912006811155C00D
:101C100062E08FE00E948C0162E083E0DF91CF916F
:101C20001F910F91FF90DF90CF90BF90AF900C94D9
:101C30008C01DF3F99F2CF3F89F2D13079F2C13088
:101C400069F28091200662EE71E0882391F261ECE6
:101C500071E080E00E94D10862ED71E089E195E0D9
:101C60000E943B2A80919C044AE06AE275E090E081
:101C70000E9413296AE275E089E195E00E94272A13
:101C800067ED71E089E195E00E94272A80919B042D
:101C90004AE06AE275E090E00E9413296AE275E08A
:101CA00089E195E00E94272A6EED71E089E195E0D7
:101CB0000E94272A69E175E09CCFDF91CF911F91A7
:101CC0000F91FF90DF90CF90BF90AF9008958F92CB
:101CD0009F92AF92BF92CF92DF92EF92FF920F93BB
:101CE0001F9310925A0580914E0590914F05A09137
:101CF0005005B0915105AC01BD01405C5F4C6A4696
:101D00007109413E53496440710518F021E0209368
:101D10005A0520915B05211104C020915A0521111B
:101D20003CC0C0900C05D0900D050D2C000CEE08A9
:101D3000FF080091360510913705012E000C220B8B
:101D4000330B8090520590905305092C000CAA0883
:101D5000BB084091580540FF2CC084519A4EA844BE
:101D6000BF4FBC01CD01600F711F821F931F680D13
:101D7000791D8A1D9B1D6C197D098E099F09009193
:101D8000F5051091F605012E000C220B330B601B9C
:101D9000710B820B930B0E94C6061F910F91FF904F
:101DA000EF90DF90CF90BF90AF909F908F900C946A
:101DB000BA0C4CEE55E167EB70E0481959096A0915
:101DC0007B090C0D1D1D2E1D3F1D800F911FA21F95
:101DD000B31F8A019B01081B190B2A0B3B0BC9017E
:101DE000B801D9CF0E94670E0E9447062091FC05DA
:101DF0003091FD05DC010E940C2A2AE030E040E031
:101E000050E00E94C12980914E0590914F05A0910C
:101E10005005B0915105821B930BA40BB50B809319
:101E2000150190931601A0931701B093180108951E
:101E30003F924F925F926F927F928F929F92AF925A
:101E4000BF92CF92DF92EF92FF920F931F93CF93A7
:101E5000DF930E949800EC0130900E0580911901EB
:101E600042E0882309F4C3C1341609F4F2C04315D3
:101E700078F181E0381609F470C081E10E943501E3
:101E8000892B09F028C281E0381640F043E0431561
:101E900008F008C284E0381609F40CC280910E05DF
:101EA0008F5F80930E0581E080931901DF91CF91C0
:101EB0001F910F91FF90EF90DF90CF90BF90AF9068
:101EC0009F908F907F906F905F904F903F9008957C
:101ED00043E0341609F445C184E03812CECF209196
:101EE0001206309113063093390520933805CE0140
:101EF00067EE7FEF0E94F22942E3469FC001479FB1
:101F0000900D1124820F931F9093490580934805EB
:101F10002091480530914905CE0169E170E00E94A9
:101F2000F22942E3469FC001479F900D1124820F82
:101F3000931F97FDABC1813D47E0940714F080EDFE
:101F400097E09093130680931206C530D1050CF0EC
:101F5000A0C1892B09F491CF43C100910C061091C7
:101F60000D061093390500933805CE01D7FD019673
:101F700095958795081B190B6091170670911806A7
:101F80008091190690911A0628EE33E040E050E067
:101F90000E94C129021B130B1093490500934805A9
:101FA00000914805109149056E01D7FF03C04FEF1E
:101FB000C41AD40AD594C79488EAC81A84EED80AF9
:101FC000C00ED11E0D2C000CEE08FF086091170604
:101FD000709118068091190690911A0628EE422EEB
:101FE00023E0522E612C712CA30192010E94C12981
:101FF00049015A01C814D904EA04FB0490F0609125
:102000001B0670911C0680911D0690911E06A3016F
:1020100092010E94C129C216D306E406F50608F40F
:10202000960130930D0620930C06C530D1050CF0B7
:10203000F0C06901F12CE12C015011098C149D04B0
:10204000AE04BF0408F019CF10934905009348056A
:1020500014CF00910E0610910F06109339050093CE
:102060003805C0900C06D0900D06F12CE12C609143
:102070001B0670911C0680911D0690911E0628EE8D
:1020800033E040E050E00E94C1292C193D094E097F
:102090005F09DE010E94B92920E034E040E050E011
:1020A0000E948F29C20ED31EE41EF51E0C191D09B5
:1020B000109349050093480560911B0670911C061A
:1020C00080911D0690911E0628EE33E040E050E01E
:1020D0000E94C12969017A0100910C0610910D0638
:1020E0004801B12CA12C281939094A095B09DE01E4
:1020F0000E94B92920E034E040E050E00E948F299E
:10210000280D391D4A1D5B1D809148059091490598
:102110002C01092E000C66087708420E531E641E1F
:10212000751E481459046A047B040CF490C0280FEF
:10213000391FC414D504E604F70408F4960130935B
:102140000F0620930E06C530D1050CF082C0019712
:102150000217130708F091CE909349058093480524
:102160008CCE2091100630911106309339052093C2
:102170003805CE016BEF7FEF0E94F22942E3469FC4
:10218000C001479F900D1124820F931F9093490522
:10219000809348052091480530914905CE0165E0BE
:1021A00070E00E94F22942E3469FC001479F900DD4
:1021B0001124820F931F823391050CF459C0813191
:1021C00047E2940714F080E197E290931106809320
:1021D0001006C530D1050CF04EC0C29709F44DCEA3
:1021E00022533109309349052093480546CE3416D1
:1021F00009F462CF431528F081E0381609F4D0CEF7
:102200003CCE43E0341631F284E0381609F480CE37
:1022100034CECD3FD3400CF430CE6901F12CE12C0B
:1022200060911B0670911C0680911D0690911E0600
:1022300028EE33E040E050E00E94C129C216D306E8
:10224000E406F50608F019CE0F5F1F4FFDCE98018A
:1022500076CFCD3FD3400CF410CEA90170E060E002
:102260004C155D056E057F0508F007CE019674CF0D
:1022700082E390E0AACFCD3FD3400CF4FECD803175
:10228000974209F4FACD2E5C3F4FACCF90E080E04E
:1022900058CECD3FD3400CF4F0CD803D974009F4AB
:1022A000ECCDF1CF41E062E370E088E592E00E947E
:1022B0008406F4CD1092690542E062E370E088E59F
:1022C00092E00E9484066DE771E081E00E94D108EF
:1022D0000E94F20EE3CD86E0809369051092190109
:1022E00042E0341609F456C04315C8F081E03816B0
:1022F000A9F169E175E081E0DF91CF911F910F9124
:10230000FF90EF90DF90CF90BF90AF909F908F9015
:102310007F906F905F904F903F900C94D10843E076
:10232000341609F443C084E03812E3CF4AE06AE28D
:1023300075E080911206909113060E9413296DE6B4
:1023400072E089E195E00E943B2A6AE275E089E14A
:1023500095E00E94272A6FE072E017C04AE06AE227
:1023600075E080910C0690910D060E94132962EF92
:1023700071E089E195E00E943B2A6AE275E089E11B
:1023800095E00E94272A69EF71E089E195E00E94BB
:10239000272AAFCF4AE06AE275E080910E0690915D
:1023A0000F060E9413296EEF71E0E3CF4AE06AE264
:1023B00075E080911006909111060E94132965E046
:1023C00072E089E195E00E943B2A6AE275E089E1CA
:1023D00095E00E94272A6BE072E0D7CFCF92DF9280
:1023E000EF92FF921F93CF93DF930E949800EC012E
:1023F00080911901882361F080910E05833009F4E2
:1024000061C0A0F5813009F447C0823009F457C09B
:1024100010910E05133009F4D1C008F073C01130CB
:1024200009F498C0123009F4B3C081E10E9435016B
:10243000892B09F0D7C1133009F4A2C108F05DC19E
:10244000113009F473C1123009F48CC180910E056A
:102450008F5F80930E0581E080931901DF91CF910A
:102460001F91FF90EF90DF90CF900895853081F11C
:1024700060F1863069F68091FE059091FF0590939A
:102480000D0580930C0590933905809338058C1BBE
:102490009D0B885C910931C08091580582608093C2
:1024A00058050E94BA0C8091160690E09093390569
:1024B00080933805D0934905C0934805A9CF8091F2
:1024C0001F06F3CF80912006F0CF8091FB05EDCF62
:1024D0002091140630911506309339052093380564
:1024E000CE0166EF7FEF0E94F2294AE0469FC001CD
:1024F000479F900D1124820F931F9093490580935D
:10250000480586CF153009F4B3C008F49BC01630D7
:1025100009F08BCF2091480530914905CE018853B1
:102520009F4F820F931F883C91050CF4DAC0813BCA
:1025300044E0940714F080EB94E09093FF058093BF
:10254000FE05C530D1050CF0CFC0883C910509F4DB
:102550006CCFB2C080914805909149059E01281B1F
:10256000390BC901049620913805309139054AE1AB
:10257000429FE001439FD00D11248C0F9D1F8F7748
:1025800099276AE170E00E94F229609316064DCF08
:102590008091480590914905C81BD90B2496C6FB2C
:1025A000CC24C0F8D12C8091380590913905C80E03
:1025B000D91E4C2D417040931F0637CF20914805FE
:1025C00030914905CE01821B930B68E270E00E94B6
:1025D000F2298091380590913905680F791F77FDB0
:1025E00015C06A31710514F069E170E0609320064E
:1025F000C530D105CCF461110BC062E08FE00E94C0
:102600008C0162E083E00E948C010FCF60E0EECF8E
:10261000265F3F4F309349052093480560E08FE0E7
:102620000E948C0160E0EECFCD3FD34044F0693191
:10263000A9F32A50310930934905209348056623B0
:10264000E1F2ECCF8091480590914905C81BD90B68
:102650002496C6FBEE24E0F8F12C80913805909189
:102660003905E80EF91E3E2D31703093FB05DDCEA5
:102670002091480530914905CE016AE070E00E9442
:10268000F2294AE0469FC001479F900D1124820F16
:10269000931F8A309105BCF0893E43E0940714F003
:1026A00088EE93E09093150680931406C530D1050B
:1026B0006CF4449708F4B9CE2A5031093093490597
:1026C00020934805B2CE8AE090E0ECCFCD3FD340D6
:1026D0000CF4ABCE883E934009F4A7CE265F3F4F63
:1026E000EDCF88EC90E029CFCD3FD3400CF49DCEC8
:1026F000803B944009F499CEF1CF153009F464C0C1
:1027000008F455C0163009F0A1CE1092690542E0D8
:1027100062E370E088E592E00E9484066DE771E074
:1027200081E00E94D1080E94F20E90CE41E062E367
:1027300070E088E592E00E94840668EC70E080E03A
:1027400090E00E94DC038091160681117FCE82E02A
:1027500080930E0580910701811178CE83E08093EC
:102760000E0574CE41E062E370E088E592E00E94DD
:10277000840668EC70E080E090E00E94DC03EACF21
:102780000E94800D41E062E370E088E592E00E94E3
:10279000840668EC70E080E090E00E94DC038091A9
:1027A0001401811153CE80910E058E5FD8CF809198
:1027B000FB05811109C08AE090E090931506809393
:1027C000140685E080930E0541E062E370E088E541
:1027D00092E00E94840668EC70E080E090E00E9445
:1027E000DC0334CE84E08093690510921901133024
:1027F00009F466C088F4113071F1123009F451C047
:1028000069E175E081E0DF91CF911F91FF90EF903A
:10281000DF90CF900C94D108153009F47BC008F4F8
:1028200070C0163069F74AE06AE275E08091FE05F3
:102830009091FF050E94132964E772E089E195E019
:102840000E943B2A6AE275E089E195E00E94272A0E
:102850006BE072E011C063E172E089E195E00E94F3
:102860003B2A809116068230B1F058F4882381F01B
:1028700067E272E0813021F689E195E00E94272A23
:10288000BFCF833059F06EE272E08430A9F3B8CF45
:1028900069E172E0F1CF62E272E0EECF63E372E0F1
:1028A000EBCF67E372E089E195E00E943B2A8091DB
:1028B0001F0669E073E08111DFCF66E174E0DCCFD1
:1028C00080912006811107C062EE71E089E195E0F8
:1028D0000E943B2A95CF64E472E080E00E94D10818
:1028E000809120064AE06AE275E090E00E94132998
:1028F00061E572E089E195E00E943B2A6AE275E0B9
:10290000BBCF6EE572E089E195E00E943B2A8091A1
:10291000FB05CFCF4AE06AE275E080911406909102
:1029200015060E94132969E672E089E195E00E948C
:102930003B2A6AE275E089E195E00E94272A60E17E
:1029400072E09ACF4F925F926F927F928F929F9296
:10295000AF92BF92EF92FF920F931F93CF93DF93AB
:102960000E949800EC0110910E05809119018823B6
:1029700049F1123009F473C0133009F479C01130F1
:1029800091F4609117067091180680911906909144
:102990001A0628EE33E040E050E00E94C12930934F
:1029A000390520933805CE01D7FD01969595879579
:1029B0002091380530913905281B390B3093490592
:1029C00020934805123009F469C0133009F414C18A
:1029D000113009F0B4C02091480530914905CE016D
:1029E000D7FD019695958795820F931F092E000CB0
:1029F000AA0BBB0BF82E092FFA2FEB2F813345E7DB
:102A00009407A105B10528F070E3F72E05E7F0E083
:102A1000E0E04F2D502F6F2F7E2F483EE3E05E0702
:102A20006105710520F448EE53E060E070E04093EA
:102A30001706509318066093190670931A06C5304E
:102A4000D105FCF4893E9340A105B10508F477C097
:102A50002A503109309349052093480570C0609190
:102A60001B0670911C0680911D0690911E0691CF49
:102A70008091FC059091FD05909339058093380570
:102A800092CFCD3FD3400CF45AC080339547A10577
:102A9000B10508F054C0265F3F4FDCCFE0904805F9
:102AA000F0904905CE01D7FD0196959587958E0D3D
:102AB0009F1D4C01990FAA08BB08609117067091E1
:102AC00018068091190690911A0628EE33E040E02E
:102AD00050E00E94C1298091FC059091FD052901DB
:102AE0003A01480E591E611C711CD301C20188169F
:102AF0009906AA06BB0608F468C021E3821625E7FA
:102B00009206A104B10430F050E3852E55E7952ECE
:102B1000A12CB12C80921B0690921C06A0921D063F
:102B2000B0921E06C530D1050CF052C04AE0E41A3E
:102B3000F10888159905AA05BB0508F458C081E17C
:102B40000E943501892B09F0A8C0123009F47FC01A
:102B5000133009F491C0113009F520911706309116
:102B600018064091190650911A06A8EEB3E00E948B
:102B7000AE296093170670931806809319069093F8
:102B80001A0641E062E370E088E592E00E94840664
:102B900068EC70E080E090E00E94DC0380910E051C
:102BA0008F5F80930E0581E080931901DF91CF91B3
:102BB0001F910F91FF90EF90BF90AF909F908F90DB
:102BC0007F906F905F904F90089542015301A2CF84
:102BD000CD3FD3400CF4B3CFE0E38E16E5E79E067D
:102BE000A104B10408F0ABCF2AE0E20EF11CF09290
:102BF0004905E0924805A3CF209148053091490549
:102C0000CE01D7FD019695958795820F931F8A3047
:102C100091058CF0853F41E0940714F084EF91E03A
:102C20009093FD058093FC05C530D1053CF40A97CF
:102C300009F485CF0DCF8AE090E0F2CFCD3FD340AD
:102C40000CF47DCF843F914009F479CF24CF2091BB
:102C50001B0630911C0640911D0650911E06A8EEE1
:102C6000B3E00E94AE2960931B0670931C0680930C
:102C70001D0690931E0685CF1092690542E062E31F
:102C800070E088E592E00E9484066DE771E081E0E3
:102C90000E94D1080E94F20E81CF83E080936905E3
:102CA000109219011230C1F1133009F445C01130EE
:102CB00009F07CCF60911706709118068091190673
:102CC00090911A062AE04AE255E00E942D296EE70B
:102CD00072E089E195E00E943B2A6AE275E089E1B1
:102CE00095E00E94272A69EF71E089E195E00E9452
:102CF000272A69E175E081E0DF91CF911F910F9163
:102D0000FF90EF90BF90AF909F908F907F906F90CB
:102D10005F904F900C94D10860911B0670911C0637
:102D200080911D0690911E062AE04AE255E00E941D
:102D30002D2963E872E0CDCF4AE06AE275E0809128
:102D4000FC059091FD050E94132968E872E0C1CF4F
:102D500080915D0591E0892780935D05811108C010
:102D600010923505109234051092370510923605F1
:102D70000E94F20E81E08093190180910B0681116F
:102D800010920B060C94BA0C1F93CF93DF930E9402
:102D9000980020916905223089F02091580520FF84
:102DA00042C02091FA0526952150330B3093390506
:102DB0002093380590934905809348052091480554
:102DC00030914905821B930B62E370E00E94F22967
:102DD000C0913805D0913905C60FD71FC370DD27C4
:102DE00021961C2F110F1093830481E10E9435015D
:102DF000892BF9F4109269058091580580FF16C05F
:102E00001093FA0542E062E370E088E592E00E94E8
:102E100084066DE771E081E00E94D108DF91CF91D7
:102E20001F910C94F20E2091F905BDCF1093F90576
:102E3000E9CF82E080936905C150C0931C010E94D4
:102E4000670E809183044AE06AE275E090E00E9498
:102E5000132962E972E089E195E00E943B2A6AE267
:102E600075E089E195E00E94272A6FE972E089E127
:102E700095E00E94272A69E175E081E0DF91CF911A
:102E80001F910C94D1088695815080931C010E945B
:102E9000670E0E94670E90910A0680915805911165
:102EA00003C0809308060895809309060895409111
:102EB0004E0550914F0560915005709151058091DC
:102EC0000B0690910A069923D1F110920A064093BD
:102ED000400550934105609342057093430540912E
:102EE0004405509145056091460570914705409312
:102EF0004E0550934F056093500570935105811115
:102F000004C080910806809358058091580580FF81
:102F100036C08091FA050E944317809167058111A0
:102F200031C080915805823068F18091FE05909102
:102F3000FF0590930D0580930C050C94F20E91E023
:102F400090930A06409344055093450560934605C7
:102F500070934705409140055091410560914205AD
:102F60007091430540934E0550934F056093500573
:102F7000709351058111C9CF80910906C4CF80910A
:102F8000F905C9CF10920D0510920C05D6CFCF923E
:102F9000DF92EF92FF920E94470620914C053091FC
:102FA0004D05821B930B97FF03C091958195910965
:102FB0000997B4F0109254051092550510925605D9
:102FC00010925705109269050E94F20E60E971E0B7
:102FD00080E090E0FF90EF90DF90CF900C94DC03C6
:102FE0008EE00E943501892B21F080915B058111D3
:102FF000E1CF81E10E943501892BE1F28091200629
:10300000882309F46AC08091200681116DC084E094
:103010000E943501892B71F20E940F04C090540563
:10302000D0905505E0905605F0905705C616D70686
:10303000E806F90608F04CC080916905853009F072
:1030400059C08091100690911106C0904E05D09005
:103050004F05E0905005F0905105C80ED91EE11CB7
:10306000F11CC0924E05D0924F05E0925005F092AF
:10307000510520910E0630910F06A8EEB3E00E9494
:10308000E3296C157D058E059F0570F420910C06D3
:1030900030910D060E94E32960934E0570934F0511
:1030A00080935005909351050E94670E0E940F0473
:1030B0002091120630911306620F731F811D911D1E
:1030C000609354057093550580935605909357056A
:1030D000FF90EF90DF90CF9008958FE00E94350130
:1030E000892B09F090CF66CF80919604882309F44C
:1030F0008ECF60CF0E945717D9CFCF92DF92EF9239
:10310000FF9280917C04811115C180912006882353
:1031100009F46DC08091200681112EC19091160690
:10312000992339F0882309F42CC18091200681115C
:103130002FC18091590581113FC0C0905405D09096
:103140005505E0905605F0905705C114D104E104EF
:10315000F10491F180916705882371F10E940F04B9
:10316000C616D706E806F90638F58091FB058823D0
:1031700019F110926705109254051092550510929E
:103180005605109257058091FE059091FF0590938A
:103190000D0580930C050E94F20E80910B068111A3
:1031A0000E94571760E087E00E945E016AE070E0CD
:1031B00080E090E00E94DC0380911606811161C1DD
:1031C00080917C04882309F44CC18091580581FFCB
:1031D00048C161E086E00E945E018091FE05909109
:1031E000FF05FF90EF90DF90CF900C94C8018FE027
:1031F0000E943501892B09F08DCF81E080937C04FA
:103200008091FB058111C9C080911606882379F150
:103210009091580591FF2BC091E090935905109221
:103220008E0410928F04109290041092910480FFEB
:10323000BAC081E091E0909306018093050180E09F
:1032400091E09093030180930201809120068823EE
:1032500009F4B2C0809120068111C3C0809120067C
:10326000882309F4C3C0809120068111D4C08091C5
:10327000670581115AC08091FB05882309F455C068
:1032800060E070E0CB010E94C60661E087E00E942A
:103290005E0181E0809367058091580590910A0650
:1032A0009111BEC080930806109235051092340526
:1032B000109237051092360510920D0510920C05EC
:1032C00061E470E080E090E00E94DC0380910B06F6
:1032D000882309F4A8C00E94571780916305909134
:1032E0006405A0916505B0916605885B9F4FAF4F5F
:1032F000BF4F8093630590936405A0936505B093D9
:10330000660580915F0590916005A0916105B0917F
:103310006205885B9F4FAF4FBF4F80935F059093CF
:103320006005A0936105B093620580917C048823B9
:1033300009F4FFCE0E940F04209114063091150667
:10334000620F731F811D911D609354057093550585
:10335000809356059093570580912006882309F4A1
:1033600065C080912006882309F4E3CE80919604FD
:10337000882309F461C0DDCE9091960491113DCF70
:10338000CDCE83E00E943501892B09F436CFCDCE16
:1033900080918904811131CFCCCE80915805826013
:1033A0008093580531CF80E091E09093060180939F
:1033B000050181E091E045CFE0910201F091030128
:1033C00080810E943501892B09F044CF0E940F04AF
:1033D000609363057093640580936505909366051B
:1033E0003DCF809196048111F1CF38CFE091050156
:1033F000F091060180810E943501892B09F033CFBD
:103400000E940F0460935F057093600580936105CF
:10341000909362052CCF809189048111F1CF27CF41
:103420008093090641CF0E94F20E57CF8FE00E9491
:103430003501892B09F495CF10927C040E940F046A
:103440002091140630911506620F731F811D911D86
:1034500060935405709355058093560590935705D6
:1034600068CE84E00E943501019759F460E086E05F
:103470000E945E0185E0FF90EF90DF90CF900C946A
:103480002204FF90EF90DF90CF9008950F931F9349
:10349000CF938091540590915505A0915605B09118
:1034A0005705892B8A2B8B2B21F08091FB058111ED
:1034B000CEC08EE00E943501892BB1F18091670565
:1034C000811132C060E070E0CB010E94C60681E04D
:1034D00080936705109235051092340510923705D8
:1034E0001092360510920D0510920C058091FB0587
:1034F000882359F0809158058D7F809358059091CD
:103500000A06911196C08093080661E470E080E09D
:1035100090E00E94DC030E94F20E0E94BA0C80919F
:103520000B0681110E9457178EE00E943501892BEE
:1035300009F08DC080916705882309F488C062E393
:1035400070E080E090E00E94DC038EE00E94350194
:10355000892B09F07CC0C0915805C23008F04DC0DD
:1035600080912106882309F448C061E087E00E9429
:103570005E0161E086E00E945E0182E999E00E94BE
:10358000C80180914E0590914F05A0915005B091D2
:1035900051050091520510915305012E000C220B8C
:1035A000330BCC2309F448C08258904EA844BF4F37
:1035B000BC01CD01600F711F821F931F0091F505A3
:1035C0001091F605012E000C220B330B601B710BC2
:1035D000820B930B0E94C6066AEF70E080E090E0D9
:1035E0000E94DC0360E086E00E945E0185E00E94AC
:1035F000220460E087E00E945E01109267050E944D
:10360000670E0E94BA0C80910B0681110E94571719
:103610008091580581FF1BC08091FE059091FF05A8
:1036200090930D0580930C05CF911F910F910C94F1
:10363000F20E8093090669CF4EE75FE167EB70E019
:10364000481B590B6A0B7B0BCB01BA01BFCFCF9143
:103650001F910F9108950F931F930E949800E0917E
:103660005805209169052130C1F02091F505309170
:10367000F605E13021F02091F7053091F8053093FF
:103680003905209338052091380530913905281BDC
:10369000390B309349052093480520914805309116
:1036A0004905AC01420F531FBA014131F7E25F07F0
:1036B00014F060E177E2603FF8ED7F0714F460EF0B
:1036C00078EDE13089F47093F6056093F505853067
:1036D00091055CF5413F584D8CF02A5031093093EB
:1036E0004905209348050AC07093F8056093F705D3
:1036F00085309105D4F4413F584D7CF781E10E941B
:103700003501892BD9F41092690542E062E370E03B
:1037100088E592E00E9484066DE771E081E00E94F6
:10372000D1081F910F910C94F20E8D3F934034F30A
:10373000403157421CF7265F3F4FD1CF809168053B
:10374000882329F080E10E943501892BE1F681E090
:103750008093690580915805813021F50E94670E9C
:103760004AE06AE275E08091F5059091F6050E94C5
:10377000132962EA72E089E195E00E943B2A6AE23D
:1037800075E089E195E00E94272A6BE072E089E10B
:1037900095E00E94272A69E175E081E01F910F9171
:1037A0000C94D108A091F705B091F80524E630E01B
:1037B0000E940C2A60547F48884D9B4C60931D01E9
:1037C00070931E0180931F019093200100914E057C
:1037D00010914F0520915005309151056CEE75E127
:1037E00087EB90E0601B710B820B930B0E94C60667
:1037F000A091F705B091F80524E630E00E940C2A6C
:103800002BE633E040E050E00E948F29CA01B90165
:103810002AE04AE255E00E941E296AEA72E089E144
:1038200095E00E943B2A6AE275E089E195E00E94FA
:10383000272A60EB72E0ABCF1F920F920FB60F9268
:1038400011242F933F938F939F93AF93BF938091B6
:103850006B0590916C05A0916D05B0916E0530914E
:103860006A0523E0230F2D3758F50196A11DB11DE0
:1038700020936A0580936B0590936C05A0936D056A
:10388000B0936E0580916F0590917005A0917105C0
:10389000B09172050196A11DB11D80936F059093A3
:1038A0007005A0937105B0937205BF91AF919F9180
:1038B0008F913F912F910F900FBE0F901F901895F1
:1038C00026E8230F0296A11DB11DD2CF1F920F92A1
:1038D0000FB60F9211242F933F934F935F936F93E3
:1038E0007F938F939F93AF93BF93EF93FF938091B9
:1038F000C3059091C405A091C505B091C605892B5B
:103900008A2B8B2BD1F19091BE05E091BF05F091F0
:10391000C0058081892780838091C3059091C4056B
:10392000A091C505B091C605181619061A061B0602
:103930009CF48091C3059091C405A091C505B091F8
:10394000C6050197A109B1098093C3059093C405E9
:10395000A093C505B093C605FF91EF91BF91AF91BC
:103960009F918F917F916F915F914F913F912F9197
:103970000F900FBE0F901F901895809123010E9409
:103980002204EACF1F920F920FB60F9211242F93A9
:103990003F934F935F936F937F938F939F93AF93D7
:1039A000BF93CF93EF93FF9396B1C0910105C0955C
:1039B00080910A058923C82390930105C0FF05C0A3
:1039C000E0911201F09113010995C1FF05C0E0914A
:1039D0000801F09109010995C2FF05C0E0910A01B3
:1039E000F0910B010995C3FF05C0E0910C01F09126
:1039F0000D010995C4FF05C0E0910E01F0910F0182
:103A00000995C5FF05C0E0911001F09111010995DC
:103A1000FF91EF91CF91BF91AF919F918F917F9146
:103A20006F915F914F913F912F910F900FBE0F902B
:103A30001F9018951F920F920FB60F9211242F937B
:103A40003F934F935F936F937F938F939F93AF9326
:103A5000BF93EF93FF938091B900887F803609F47C
:103A60004AC0F0F5883209F4A7C018F5803109F48E
:103A70009BC0B8F4882309F4F9C0883009F494C0D5
:103A8000FF91EF91BF91AF919F918F917F916F9136
:103A90005F914F913F912F910F900FBE0F901F900C
:103AA0001895883109F488C0803251F780939705C2
:103AB00014C0803409F49DC040F48033B9F38833D6
:103AC000F9F68093970585ECB0C0803509F485C080
:103AD000883509F496C0883499F60E947C04D0CFCA
:103AE000883909F48CC038F5883729F050F48836C5
:103AF00011F0803729F683E0809399051092FF0436
:103B000057C0883809F47BC0803919F0803809F033
:103B1000B7CF8091FF04803208F071C0E091FF04BC
:103B200081E08E0F8093FF048091BB00F0E0E152B2
:103B3000FB4F80833DC0803B39F0E0F4803A09F4CC
:103B400079C0883A09F09CCF84E08093990510925F
:103B5000DE041092DD04E0910505F091060509955B
:103B60008091DD0481110FC081E08093DD0410920B
:103B7000BD0409C0803C09F4A6CF883C09F4A3CF5A
:103B8000883B09F07DCFE091DE0481E08E0F8093C9
:103B9000DE04F0E0E354FB4F80818093BB00909102
:103BA000DE048091DD0429C0809174058093BB0000
:103BB00085EC8093BC0064CF90919605809195052B
:103BC000981758F5E091960581E08E0F8093960541
:103BD000F0E0EB58FA4F8081E9CFE091960581E063
:103BE0008E0F809396058091BB00F0E0EB58FA4F62
:103BF000808390919605809195059817C8F285E885
:103C0000D8CFE091960581E08E0F80939605809144
:103C1000BB00F0E0EB58FA4F80838091980581114A
:103C20005CCF81E08093730584EA8093BC0010929E
:103C3000990526CF85EC8093BC0010929905809160
:103C4000FF04803230F4E091FF04F0E0E152FB4FDA
:103C500010826091FF0470E0E0910305F09104058B
:103C60008FED94E009951092FF040ACF109297050A
:103C700034CFEFECF5E01382128288EE93E0A0E0FF
:103C8000B0E084839583A683B78388E291E0918333
:103C90008083E3EFF5E080E181838CED95E0938311
:103CA000828387E296E09583848384E0868388E03C
:103CB000878391E0908722E330E03287218720E2FA
:103CC00033E03487238748E058EB6CE670E04587A3
:103CD00056876787708B418B528B638B748B158AE9
:103CE000168A178A108E2CEB3BE1328F218F2EEE35
:103CF0003BE1348F238F28EE33E0368F258F24EF7E
:103D000031E030A3278F2EE531E032A321A313A2A7
:103D100040EC5FEC6AE670E044A355A366A377A38A
:103D200040EA53E66FE670E040A751A762A773A789
:103D300014A615A616A6EBEDF5E0138212822AE36F
:103D400031E03183208384838FEF858389E086830C
:103D50008AE087838BE080878CE081878DE0828793
:103D60001386148615861686178681E00C9425081E
:103D7000CF93DF93CDB7DEB728970FB6F894DEBFA9
:103D80000FBECDBF789484B5826084BD84B5816058
:103D900084BD85B5826085BD85B5816085BD809116
:103DA0006E00816080936E0010928100809181008E
:103DB0008260809381008091810081608093810086
:103DC000809180008160809380008091B100846048
:103DD0008093B1008091B00081608093B0008091A9
:103DE0007A00846080937A0080917A008260809368
:103DF0007A0080917A00816080937A0080917A00C5
:103E0000806880937A001092C1008DE18093F30561
:103E100065EB72E089E195E00E943B2A82E00E9416
:103E2000250881E08093220162E081E10E948C01FB
:103E300062E080E10E948C0162E084E00E948C01DB
:103E400062E08EE00E948C0162E087E00E948C01BB
:103E500064E670E080E090E00E94DC0387E00E946E
:103E60003501892B51F0109214011092FB058AE064
:103E700090E0909315068093140661E087E00E941D
